:020000021000EC
:10F800000C9446FC0C9463FC0C9463FC0C9463FC19
:10F810000C9463FC0C9463FC0C9463FC0C9463FCEC
:10F820000C9463FC0C9463FC0C9463FC0C9463FCDC
:10F830000C9463FC0C9463FC0C9463FC0C9463FCCC
:10F840000C9463FC0C9463FC0C9463FC0C9463FCBC
:10F850000C9463FC0C9463FC0C9463FC0C9463FCAC
:10F860000C9463FC0C9463FC0C9463FC0C9463FC9C
:10F870000C9463FC0C9463FC0C9463FC0C9463FC8C
:10F880000C9463FC0C9463FC0C9463FC11241FBE69
:10F89000CFEFD0E1DEBFCDBF11E0A0E0B1E0E4E604
:10F8A000FFEF01E00BBF02C007900D92A030B1073F
:10F8B000D9F712E0A0E0B1E001C01D92A434B10775
:10F8C000E1F70C9474FF0C9400FC0F92AF93BF937C
:10F8D000CF93DF93EF93FF93FC01EA01DB01D8950F
:10F8E000099231961197D9F7FF91EF91DF91CF915E
:10F8F000BF91AF910F9008950F921F920F93AF9306
:10F90000BF93CF93DF93EF93FF93FC01EA01DB01F9
:10F910000990199001E043D032961297C9F7FC0183
:10F9200003E03DD005E03BD0FF91EF91DF91CF9117
:10F93000BF91AF910F911F900F9008950F931F9358
:10F94000EF93FF93FC0103E02AD000E011E0E00F09
:10F95000F11FE617F707B9F7FF91EF911F910F918C
:10F9600008950F930F9222D0082E09E018D00F901F
:10F970000F9108950F930F92EF93FF9317D0FC010F
:10F9800060936800C895802DFF91EF910F900F91C3
:10F9900008950F930BD001E102D00F910895E199E2
:10F9A000FECF00936800E895FFFF0000009168001B
:10F9B00000FDFCCF089583E08093990080919A0028
:10F9C000886180939A00089580919A00877E809341
:10F9D0009A00089580939C0080919B0086FFFCCF45
:10F9E00080919B00806480939B00089580919C008F
:10F9F0009927089580919B009927807890700895A9
:10FA0000EF92FF920F931F93CF93DF937B01C0E0A0
:10FA1000D0E0C617D70770F48C010E94FAFC882347
:10FA2000E1F30E94F6FCF80181938F012196CE1537
:10FA3000DF0598F381E090E0DF91CF911F910F9166
:10FA4000FF90EF900895EF92FF920F931F93CF9343
:10FA5000DF937C018B01C0E0D0E0C017D10738F400
:10FA6000F70181917F010E94EAFC2196F6CF81E0A7
:10FA700090E0DF91CF911F910F91FF90EF9008954B
:10FA800040E050E04817590750F42AE633E0000000
:10FA90002150304037FFFBCF4F5F5F4FF3CF0895CA
:10FAA0000E94E4FC0E94000008950E94FAFC882352
:10FAB000E1F30E94F6FC803219F481E090E00895B1
:10FAC00085E10E94EAFC80E090E0089590E0282F14
:10FAD00033272138310589F02238310524F42038C4
:10FAE000310549F00DC02238310549F0283931057A
:10FAF00039F493E005C092E003C091E001C092E1C7
:10FB0000892F9927089540E050E06091400170915D
:10FB1000410146175707D0F4209142023091430229
:10FB2000E2E4F1E03FBB2EBB2F5F3F4F80818DBBF6
:10FB3000E29AE19AE199FECF4F5F5F4F3196461707
:10FB4000570780F33093430220934202089540E028
:10FB500050E0609140017091410146175707B0F4A1
:10FB60002091420230914302E2E4F1E03FBB2EBB20
:10FB70002F5F3F4FE09A8DB381934F5F5F4F4617E2
:10FB80005707A0F330934302209342020895CF9386
:10FB9000DF93809142029091430297FF03C081E07E
:10FBA0008BBF01C01BBEC0E0D0E0809140019091AE
:10FBB0004101C817D907A0F4CE018E5B9E4F20915A
:10FBC000420230914302220F331FAC0160E071E02A
:10FBD000C9018C0F9D1F0E947CFCC050DF4FE5CFF8
:10FBE0000E94C9FCDF91CF9108952091420230918B
:10FBF000430237FF03C081E08BBF01C01BBE42E45C
:10FC000051E06091400170914101C901880F991F35
:10FC10000E9465FC0895CF93C0E069E081E090E028
:10FC20000E94BAFC992784FF03C08F7E0E94B1FC1A
:10FC30000E94FAFC8823E1F30E94F6FC99278235A2
:10FC400091051CF5803591050CF05CC0813491055F
:10FC500009F462C0823491057CF481339105B1F1DD
:10FC60008233910524F4C09709F44CC037C1803425
:10FC7000910509F437C132C18234910509F45FC09E
:10FC80008534910509F45EC029C18635910509F4D2
:10FC9000F0C0873591054CF48235910509F45FC0B9
:10FCA0008535910509F468C019C18437910509F4B7
:10FCB000A3C0853791052CF48436910509F475C0ED
:10FCC0000DC18537910509F4C4C008C10E9455FDD6
:10FCD000882309F4ADCF84E10E94EAFC81E40E940C
:10FCE000EAFC86E50E94EAFC82E50E94EAFC80E2EA
:10FCF0000E94EAFC83E50E94EAFC84E50E94EAFC9B
:10FD00008BE406C00E9455FD882309F491CF84E15D
:10FD10000E94EAFC80E1E3C061E070E080E091E0F5
:10FD20000E9400FD0E9455FD882309F481CF84E1E3
:10FD30000E94EAFC809100010E9466FDE9CF64E127
:10FD400070E008C061E070E080E091E00E9400FD9A
:10FD500064E070E080E091E00E9400FDD3CF0E945B
:10FD600055FD882309F464CF60E070E0CB010E9468
:10FD70009EFC0E94C9FCCBCF62E070E080E091E085
:10FD80000E9400FD0E9455FD882309F451CF209167
:10FD90000001809101019927982F8827820F911DDA
:10FDA0009093430280934202B2CF63E070E080E020
:10FDB00091E00E9400FD20910101809100019927AE
:10FDC000982F8827820F911D9093410180934001C5
:10FDD000BC0182E491E00E9400FD0E9455FD882351
:10FDE00009F426CF80910201863419F40E94C7FDE0
:10FDF0008ECF0E9483FD8BCF63E070E080E091E0C6
:10FE00000E9400FD20910101809100019927982F07
:10FE10008827820F911D90934101809340010E9499
:10FE200055FD882309F404CF80910201863419F42A
:10FE30000E94F5FD02C00E94A7FD84E10E94EAFC39
:10FE4000609140017091410182E491E00E9423FDA4
:10FE500061CF0E9455FD882309F4EACE84E10E9417
:10FE6000EAFC8EE10E94EAFC87E90E94EAFC82E05B
:10FE70004FCF64E070E080E091E00E9400FD0E94BE
:10FE800055FD882309F4D4CE84E10E94EAFC8091D8
:10FE90000001803531F480910101882361F4C82F7D
:10FEA00017C0883531F480910101883061F4C3E0D6
:10FEB0000FC0803531F480910101883049F4C2E0EF
:10FEC00007C0883529F480910101882309F4C1E035
:10FED00069E08C2F99270E94BAFC1ACF85E10E9415
:10FEE000EAFCA6CECF910895CFEFD0E1DEBFCDBF23
:10FEF000CEE1F894AEEFBFE00E94A9FF802D843BD5
:10FF000079F4AFEFBFE00E94A9FF802D833C41F45C
:10FF1000ADEFBFE00E94A9FF802D992780936F006D
:10FF20000E94DBFC0E94F6FC84E690E00E9440FD0B
:10FF30000E94FAFC882319F00E940BFE04C0C150F5
:10FF4000C8BBCC2389F70E9450FD80E090E00C9460
:10FF5000B1FFE199FECFBFBBAEBBE09A11960DB2E7
:04FF60000895FFCF32
:040000031000F800F1
:00000001FF
